:100000000C9446000C9463000C9463000C94630001
:100010000C9463000C9463000C9463000C946300D4
:100020000C9463000C9463000C9463000C946300C4
:100030000C9463000C9463000C9463000C946300B4
:100040000C9469010C9463000C94A4010C94CC01F1
:100050000C9463000C9463000C9463000C94630094
:100060000C9463000C9463000C9463000C94630084
:100070000C9463000C9463000C9463000C94630074
:100080000C9463000C9463000C94630011241FBE55
:10009000CFEFD0E1DEBFCDBF11E0A0E0B1E0E8E7F7
:1000A000FFE000E00BBF02C007900D92A437B1073C
:1000B000D9F712E0A4E7B1E001C01D92AE38B10754
:1000C000E1F70C9465000C940000CFEFD0E1DEBFA7
:1000D000CDBFC0E0D0E00E945702AE016EE072E0FA
:1000E00083EF91E00E94810280E091E00E94DF02B4
:1000F00088E091E00E94DF0283E291E00E94DF024B
:100100008FEF9FEF909381008093800088EB9BE0BE
:10011000909387008093860090938500809384005D
:10012000D0938900C093880082E080938B008AE19D
:1001300080938A0080918B00806880938B008091EF
:100140008B00806280938B00139A149A80E00E9447
:1001500013018093780181E00E941301282F80937E
:100160007901809178019DE7899FA001112434E0F5
:10017000569547953A95E1F74C505E4F299F90016F
:10018000112484E0369527958A95E1F72C503E4F4F
:10019000CA01840F951F9093870080938600C90140
:1001A000820F931F90938500809384008091740147
:1001B0009091750183709070892B71F58091650025
:1001C00090E18927809365003F932F938091790177
:1001D00099279F938F935F934F93809178019927ED
:1001E0009F938F93FE01E65DFE4F8081992787FDE7
:1001F00090959F938F938FE291E09F938F930E94AE
:10020000CA022196C370D0708DB79EB70C960FB6F8
:10021000F8949EBF0FBE8DBF0E9498010E94980166
:100220000E94980193CF806287B9369A3699FECFA3
:1002300085B199270895009731F0A4E0B0E01197B7
:10024000F1F70197D1F70895009731F0A0EABFE0E8
:100250001197F1F70197D1F70895CF93C82F88230D
:1002600031F084E690E00E941B01C150D1F7CF919C
:100270000895CF93C82F882331F08AE090E00E9440
:100280001B01C150D1F7CF910895CF93C82F882378
:1002900031F084E690E00E942401C150D1F7CF9163
:1002A0000895CF93C82F882331F08AE090E00E9410
:1002B0002401C150D1F7CF910895CF93C82F88233F
:1002C00031F081E090E00E942401C150D1F7CF913C
:1002D00008951F920F920FB60F9211248F939F9340
:1002E00080917601909177010196909377018093A8
:1002F00076010A976CF01092770110927601809146
:100300007401909175010196909375018093740129
:1003100086E082BF9F918F910F900FBE0F901F902C
:10032000189584E083BF12BE81E087BF789408955A
:100330002091740130917501809174019091750143
:1003400082179307C9F308951F920F920FB60F9269
:1003500011242F938F939F93EF93FF932CB1809150
:10036000030290910202891B803861F080910302A0
:10037000E82FFF27EF77F070EE5FFD4F22838F5F4E
:1003800080930302FF91EF919F918F912F910F9096
:100390000FBE0F901F9018951F920F920FB60F92DD
:1003A00011248F939F93EF93FF93909181018091FC
:1003B0008001981711F455980DC080918001E82FA5
:1003C000FF27EF77F070E058FE4F8F5F809380013A
:1003D00082818CB9FF91EF919F918F910F900FBE09
:1003E0000F901F901895CF93C82F8A3019F48DE085
:1003F0000E94F30141E050E08BB1992725E09695EA
:1004000087952A95E1F7842795279C012170307004
:1004100080FDF2CFCCB9C901CF910895CF93DF937E
:1004200090910302809102029817D1F38091020209
:10043000E82FFF27EF77F070EE5FFD4F9281C92F15
:10044000DD278F5F80930202CD30D10511F4CAE021
:10045000D0E08C2F0E94F301CE01DF91CF9108955F
:10046000CF93DF93EC018881882361F088818A3003
:1004700019F48DE00E94F30189910E94F3018881B3
:100480008823A1F7DF91CF9108950F931F93CF9306
:10049000C62F8C01662339F0F80181918F010E94EB
:1004A000F301C150C9F7CF911F910F9108959FEFAC
:1004B0009BBB1ABA98BB80E187BB95BB14BA92BBB1
:1004C00011BA93B912B81092620010926100909321
:1004D000650088E18093640010BE1092900089E16D
:1004E00089B91BB888E98AB98EE08093950087ECBA
:1004F00086B986B1877C11F03699FECF0E949101B2
:1005000008950F931F93CF93DF938C01EB01009716
:10051000A1F16CE070E081E090E00E941406FC0123
:10052000892B21F1209751F0C287D38721E02383C3
:100530008091840290918502892BD1F001151105DB
:10054000A9F000871187038102600383A0918602CE
:10055000B0918702AB2B51F4F0938702E0938602AF
:10056000C0918802D0918902CD2B51F0CF010DC0EE
:10057000F0938502E0938402E1CF672B51F605C02A
:10058000F0938902E0938802F1CFDF91CF911F9120
:100590000F910895CF93DF93CDB7DEB7E5E0F0E09C
:1005A000EC0FFD1F81919191AF01BC0180918602FA
:1005B000909187020E941703DF91CF9108950F93C6
:1005C0001F93CF93DF93DC0100E010E0E0918602FF
:1005D000F0918702838181FF23C08D91ED018823F3
:1005E00029F413C0E0918602F09187020084F1851E
:1005F000E02D0995892B11F00FEF1FEF89918823CA
:1006000089F7E0918602F09187020084F185E02D60
:100610008AE00995892B11F00FEF1FEFC80102C086
:100620008FEF9FEFDF91CF911F910F9108952F9240
:100630003F924F925F926F927F928F929F92AF9272
:10064000BF92CF92DF92EF92FF920F931F93CF93BF
:10065000DF93CDB7DEB762970FB6F894DEBF0FBE5B
:10066000CDBFAA24BB2465014C011B014D875E87C9
:1006700044245524FC0146825782838181FDACC20B
:100680008FEF9FEFB8C20894211C311C40FE92C22C
:10069000862D80538A30F0F4F0E36F1651F42A89E6
:1006A000222339F443FC05C080E091E0482A592A0E
:1006B00093C28AE09A89989F902D1124892F860DE4
:1006C00080538A8B882314F4EFE7EA8B43FC84C2BF
:1006D0007A8882C243FE05C0FA89FF2311F421E023
:1006E0002A8B862D992787FD9095883691057CF574
:1006F000853691050CF070C08335910509F49FC0D3
:1007000084359105BCF48B32910509F447C08C32D5
:10071000910544F48032910509F444C0839709F4AB
:100720004BC03EC28D32910509F441C08E9709F449
:1007300048C036C28336910509F458C08436910505
:100740000CF09AC08835910509F4D1C029C28037D0
:10075000910509F4C4C08137910584F48C36910564
:10076000B1F18D3691052CF48936910509F484C0D8
:1007700017C28F36910509F4AFC012C285379105B3
:1007800009F4B7C08637910524F483379105B9F190
:1007900007C28837910509F4AAC002C280E190E03F
:1007A000482A592AE0E2F0E04E2A5F2A15C220E8E2
:1007B00030E0422A532A10C280E490E0482A592AA5
:1007C0000BC2E8E0F0E04E2A5F2A1A8A05C224E054
:1007D00030E0422A532A00C20F2EFFE3AF2EF02D45
:1007E0007A940F2EF3E66F2EF02D65C1ED85FE8510
:1007F000CF0102968D879E87A0807A945CC1ED859B
:10080000FE859F012E5F3F4F2D873E87A080B180E0
:1008100043FE0BC03A89832F992787FD9095BC0131
:10082000C5010E9484078F8707C0F5010190002051
:10083000E9F73197EA19EF878F85781A3CC1ED8582
:10084000FE859F012E5F3F4F2D873E87A080B180A0
:1008500043FE0BC03A89832F992787FD9095BC01F1
:10086000C5010E948F078F8704C0C5010E947B07C6
:100870008F878F85781A1FC142FE0CC0ED85FE85DB
:100880009F012C5F3F4F2D873E8720813181428120
:1008900053810DC0ED85FE85CF0102968D879E8721
:1008A000808191819C01442737FD4095542F590147
:1008B0006A01552364F4E2E0F0E04E2A5F2AD09406
:1008C000C094B094A094A11CB11CC11CD11C2FEBEE
:1008D0003FEF422253222CC038E03F870AC080E419
:1008E00090E0482A592A0F2EF8E76F2EF02D90E15C
:1008F0009F8742FE0CC0ED85FE859F012C5F3F4F18
:100900002D873E8720813181428153810BC0ED8547
:10091000FE85CF0102968D879E87808191819C0103
:100920004427552759016A01EFECFFEF4E225F2261
:100930009E012F5F3F4F288B398B3F85E32EFF248D
:1009400000271127C601B501A80197010E949A0747
:10095000DC01CB01E889F98980838A301CF0860D9F
:10096000815204C0E889F9898081805DE889F9892C
:100970008193E88BF98BC601B501A80197010E940C
:100980009A0759016A012115310541055105D1F632
:10099000CE010196A888A81AC20182739070892B93
:1009A00009F07A9446FE0FC0872D992787FD909510
:1009B000FF85F03131F40F2EFEEF7F2EF02D780EF3
:1009C00002C0782E7A9443FE12C08A89282F3327DA
:1009D00027FD30958A2D9927821793072CF0E7EF92
:1009E000FFEF4E225F2203C0FA89FA19FA8B43FE09
:1009F00003C02A89721A01C07A18C20180789170E6
:100A0000892B69F4872D7A9418164CF4B40180E28E
:100A100090E00E943006872D7A941816BCF341FEB0
:100A200006C0B4018DE290E00E9430060FC044FE83
:100A300006C0B4018BE290E00E94300607C045FE7C
:100A400005C0B40180E290E00E94300646FE0FC06F
:100A5000B40180E390E00E9430063F85303139F4E4
:100A6000B401862D992787FD90950E943006852D2B
:100A7000992780FF0DC0872D7A9418164CF4B40185
:100A800080E390E00E943006872D7A941816BCF31C
:100A900043FE11C08A89982F91509A8B18165CF4E6
:100AA000B40180E390E00E9430068A89E82FE1508B
:100AB000EA8B1816ACF347FC0DC0872D7A941816F4
:100AC0004CF4B40180E290E00E943006872D7A94C5
:100AD0001816BCF3F3E66F1641F48A2DB40199277A
:100AE00087FD90950E9430064BC023E76216B9F44B
:100AF0003F8531503F873F3F09F442C0F501808177
:100B00000894A11CB11CB401992787FD90950E94FF
:100B100030068F8581508F878F3F81F731C093E5F5
:100B20006916A1F4EF85E150EF87EF3F49F1F50138
:100B30008491B40199270E9430060894A11CB11C2D
:100B4000FF85F150FF87FF3F91F71AC0CE01019654
:100B5000288939898217930799F08E010F5F1F4FFB
:100B6000E889F9898291E88BF98BB401992787FD8F
:100B700090950E943006288939890217130781F75A
:100B800047FE15C0872D7A9418168CF4B40180E2C4
:100B900090E00E943006872D7A941816BCF307C0A7
:100BA000B401862D992787FD90950E943006442434
:100BB000552412C035E2631641F44424552443946D
:100BC0001A8A7A888AE08F8707C0B401862D992710
:100BD00087FD90950E943006F401838183FF03C056
:100BE000F101649002C0F1016080662009F04BCDF4
:100BF000F4018681978162960FB6F894DEBF0FBE2E
:100C0000CDBFDF91CF911F910F91FF90EF90DF90BB
:100C1000CF90BF90AF909F908F907F906F905F909C
:100C20004F903F902F9008950F931F93CF93DF9392
:100C3000869F8001879F100D969F100D1124C8017B
:100C40000E946306EC01009729F0A80160E070E0C3
:100C50000E947407CE01DF91CF911F910F910895EB
:100C60000F931F93CF93DF938C01EB018B81992717
:100C700081FF22C082FF14C02E813F818C819D8123
:100C8000281739073CF4E881F9810193E883F98357
:100C90002E813F812F5F3F4F2E833F83C8010EC0BF
:100CA000E885F985802F0995892B31F4AE81BF81C4
:100CB0001196AE83BF83F2CF8FEF9FEFDF91CF917D
:100CC0001F910F910895CF93DF939C01029710F429
:100CD00022E030E040E050E060918C0270918D02A3
:100CE000FB01DA016115710569F18081918182173B
:100CF000930709F452C02817390738F441155105F4
:100D000019F08417950708F4AC01DF010280F38124
:100D1000E02D309751F741155105A1F0DA01A21BE2
:100D2000B30B149708F443C0DB010AC06D917C91AA
:100D300011976417750709F450C0FD01A281B381B2
:100D40001097A1F7E0918A02F0918B02309741F45D
:100D5000E0917001F0917101F0938B02E0938A02AF
:100D600040916E0150916F014115510529F14E1BC3
:100D70005F0B42175307E8F0C9010296481759075D
:100D8000C0F0EF01C20FD31F2296D0938B02C09305
:100D90008A0221933193CF0142C01097B1F0828132
:100DA0009381ED018A839B83CF01029638C09A011B
:100DB000BBCF80E090E033C04DB75EB7A091720129
:100DC000B09173014A1B5B0BD2CF228133813093E8
:100DD0008D0220938C02CF01E8CF2417350761F0F4
:100DE000EA01C21BD30BFD01EC0FFD1F21933193D0
:100DF0002297CD93DC93CFCF309741F0ED014A811C
:100E00005B8142835383CD01029609C0FD0182813B
:100E1000938190938D0280938C02CD01F5CFDF9169
:100E2000CF910895CF93DF93009709F45AC0DC0166
:100E30001297ED011A821B8280918C0290918D0293
:100E40000097D9F1FC0140E050E0EA17FB0748F4B5
:100E5000AF010280F381E02D3097A1F0EA17FB0784
:100E6000B8F3ED01EA83FB832D913C911197E901E1
:100E7000CA0FDB1FCE0102968E179F0719F141158D
:100E80005105D9F0EA01AA83BB83CA0102962881E1
:100E90003981820F931F8A179B0719F56D917C91F9
:100EA0001197260F371F2E5F3F4F28833983FD018F
:100EB000428153814A835B8314C0B0938D02A09317
:100EC0008C020FC06A817B81260F371F2E5F3F4F38
:100ED0002D933C93119722813381FD01228333832B
:100EE000CECFDF91CF910895DC0101C06D934150C9
:100EF0005040E0F70895FC0105900020E9F7809547
:100F000090958E0F9F1F0895FC01615070400190D5
:100F10000110D8F7809590958E0F9F1F0895FC01C2
:100F20006150704005900110D8F7809590958E0F14
:100F30009F1F0895A1E21A2EAA1BBB1BFD010DC025
:100F4000AA1FBB1FEE1FFF1FA217B307E407F50779
:100F500020F0A21BB30BE40BF50B661F771F881F55
:100F6000991F1A9469F760957095809590959B01EB
:080F7000AC01BD01CF010895A1
:100F78000A0A2A2A2A2A2A002A2A2A2A2A205369D5
:100F88006D706C652D536572766F2070726F677225
:100F9800616D002A2A2A2A2A0A002F2D5C7C002546
:100FA8006320536572766F31206164633A2025337C
:100FB800642070756C73653A20253464202053656D
:100FC80072766F32206164633A202533642070752D
:100FD8006C73653A20253464202020200D00000021
:040FE8008E02200055
:00000001FF
